:1000000050C0000068C0000066C0000064C000006E
:1000100062C0000060C000005EC000005CC0000064
:100020005AC0000058C0000056C0000054C0000074
:1000300052C0000050C000004EC000004CC0000084
:100040004AC0000048C0000046C0000044C0000094
:1000500042C0000040C000003EC000003CC00000A4
:100060003AC0000002C5000036C0000034C00000E5
:1000700032C0000030C000002EC000002CC00000C4
:100080002AC0000028C0000026C0000024C00000D4
:1000900022C0000020C000001EC000001CC00000E4
:1000A0005D0511241FBECFEFCDBFDFE3DEBF2CE324
:1000B000A0E0BCE301C01D92A838B207E1F710E050
:1000C000C1E5D0E003C02197FE01E7D7C035D107D5
:1000D000D1F704D5FDC794CF00008093C408809168
:1000E000C30887FFFCCF8091C4080895CF93DF93A6
:1000F00090E0FC01E55AFE4A20812F3F61F0FC01AF
:10010000EE5CFE4AE08130E2E39FF0011124FC5FE7
:10011000613021F42183DF91CF910895875F9E4A5A
:10012000EC01A881AF3F69F0CF014096A80FB92F2D
:10013000B11D9FB7F89422838C9188608C939FBFE8
:10014000EACFB0E0A0E0F5CF8091473C811117C025
:100150001092483C1092493C10924A3C10924B3C01
:1001600010924C3C10924D3C10924E3C10924F3CE1
:100170001092503C1092513C81E08093473C80911A
:10018000E3058C7F9091463C892B8093E305911188
:1001900019C061E084E0AADF61E086E0A7DF80911A
:1001A000C10884608093C1088091C00881628093F7
:1001B000C0089091403C8091413C9093C00880934E
:1001C000C1080895913031F461E08EE08FDF61E085
:1001D00080E1E4CF923019F761E08EE187DF61E0E2
:1001E00080E2DCCF90E0FC01E052FF4AE081EE23A8
:1001F00019F1E13021F000F1E630A8F00895875FB1
:100200009E4AFC012081233008F02F5F3091010AC3
:1002100081E090E001C0880F2A95EAF7809583235A
:100220008093010A089580E1E89FF0011124E05ACB
:10023000F54F81818F7E818308950F931F93CF9314
:10024000DF93C82FD0E0FE01E55AFE4A00810F3F40
:1002500099F0162F893208F4C5DFFE01EE5CFE4AE4
:10026000E08180E2E89FF0011124FC5F808180231F
:1002700051F0111106C00683DF91CF911F910F91AC
:1002800008950583F9CFC75FDE4A8881309771F002
:100290008F3F61F07096E80FF11D9FB7F894808151
:1002A000111107C0877F80839FBFE6CFF0E0E0E0B9
:1002B000F4CF8860F8CF8F929F92AF92BF92CF9287
:1002C000DF92EF92FF920F93CF93DF938091813C67
:1002D000893210F461E0B1DF8091483C882319F045
:1002E00081FF0DC07894DF91CF910F91FF90EF9037
:1002F000DF90CF90BF90AF909F908F90089580FF38
:10030000F2CF80904A3C90904B3CA0904C3CB090F7
:100310004D3CC12CD12C7601E0E09401A501B60141
:10032000C701A0E0AED681F1217030E040E050E09E
:1003300060E070E080E090E0A4D6D1F0B0E0A0E012
:10034000E03370F4AE2FA695A695A69580E2A89FFF
:10035000D0011124A05FBB4F8E2F8770A80FB11D55
:10036000CE2FD0E0CE5BD34C88899C91892B8C9387
:100370009401A501B601C70101E068D649015A01FF
:100380006B017C01EF5FC9CF80904E3C90904F3C59
:10039000A090503CB090513CC12CD12C7601E0E2B1
:1003A0009401A501B601C701A0E06BD609F49BCF6B
:1003B000217030E040E050E060E070E080E090E0EC
:1003C00060D6D1F0B0E0A0E0E03370F4AE2FA69597
:1003D000A695A69580E2A89FD0011124A05FBB4FEF
:1003E0008E2F8770A80FB11DCE2FD0E0CE5BD34CDF
:1003F00088899C91892B8C939401A501B601C70132
:1004000001E024D649015A016B017C01EF5FC8CF9E
:100410008FB7F89420912B3C30912C3C40912D3C8F
:1004200050912E3CE091AA0AF091AB0A9091A60A55
:1004300090FF08C02F5F3F4F4F4F5F4FE091AA0AD8
:10044000F091AB0A8FBFA8EEB3E0F4D523E0F695A8
:10045000E7952A95E1F76E0F7F1F811D911D089585
:100460008F929F92AF92BF92CF92DF92EF92FF92C4
:100470004B015C01CDDF6B017C01A8EEB3E0A5016F
:100480009401D8D5C60ED71EE81EF91EC616D7068B
:10049000E806F90610F4BCDFF9CFBADF6C157D056C
:1004A0008E059F05D0F3FF90EF90DF90CF90BF9027
:1004B000AF909F908F9008950F931F93CF93FC015F
:1004C000808191818831910541F48EB182FB88272A
:1004D00080F9CF911F910F9108958531910529F4ED
:1004E0008AB1881F8827881FF4CF8731910521F4AE
:1004F0008EB186958170EDCF8631910519F48EB15C
:100500008170E7CF8C31910529F48EB186FB882765
:1005100080F9DFCF8B31910529F48EB185FB8827D7
:1005200080F9D7CF8A31910521F48EB182958170FF
:10053000D0CF8931910529F48EB183FB882780F9CA
:10054000C8CF8932B0F48C011127F801E55AFE4A70
:10055000C081CF3F71F046DEF801EE5CFE4AE081DB
:1005600080E2E89FF0011124FC5F8085C82381E0D0
:1005700039F680E0C5CF8F929F92AF92BF92CF9213
:10058000DF92EF92FF920F93CF93DF938091483CDD
:10059000882319F081FF19C0F89481E38093C00883
:1005A00084E08093C1088091813C893208F098C032
:1005B00060E0DF91CF910F91FF90EF90DF90CF90AF
:1005C000BF90AF909F908F9038CE80FFE6CF809005
:1005D0004A3C90904B3CA0904C3CB0904D3CC12C80
:1005E000D12C7601E0E09401A501B601C701A0E09D
:1005F00048D589F1217030E040E050E060E070E0E3
:1006000080E090E03ED5D9F0B0E0A0E0E03370F4B7
:10061000AE2FA695A695A69580E2A89FD00111249D
:10062000A05FBB4F8E2F8770A80FB11DCE2FD0E0DB
:100630008C91CE5BD34C888B8C91887F8C9394016A
:10064000A501B601C70101E001D549015A016B01BD
:100650007C01EF5FC8CF80904E3C90904F3CA090C3
:10066000503CB090513CC12CD12C7601E0E2940179
:10067000A501B601C701A0E004D509F48ECF217011
:1006800030E040E050E060E070E080E090E0F9D4DD
:10069000D9F0B0E0A0E0E03370F4AE2FA695A695B7
:1006A000A69580E2A89FD0011124A05FBB4F8E2F9A
:1006B0008770A80FB11DCE2FD0E08C91CE5BD34CAC
:1006C000888B8C91887F8C939401A501B601C7011A
:1006D00001E0BCD449015A016B017C01EF5FC7CF37
:1006E000DF91CF910F91FF90EF90DF90CF90BF906F
:1006F000AF909F908F900895FF920F931F93CF9389
:10070000DF93C82FF62E172F042F35DF82E0E4DCAD
:100710008C2FE2DCCF2DD12F0C0F1D2F111DC017F8
:10072000D10719F08991D8DCFACFDF91CF911F91D1
:100730000F91FF90C0CD1F93CF93DF93182FD62F2B
:10074000C42F19DF85E0C8DC812FC6DC8D2FC4DC07
:100750008C2FC2DCDF91CF911F91ADCDCF93C82FED
:100760000ADF83E0B9DC8C2FB7DC80E0B5DCC82F72
:10077000A2DD8C2FCF910895CF92DF92EF92FF925E
:10078000CF93C82F482F60EE8FE0D5DF8FB7F89456
:10079000C0902B3CD0902C3CE0902D3CF0902E3C17
:1007A0008FBF8AE0C80ED11CE11CF11C2FB7F89452
:1007B00080912B3C90912C3CA0912D3CB0912E3CF3
:1007C0002FBF8C159D05AE05BF0578F48EE0C6DF02
:1007D000807EC813EBCF81E091E0892790E0CF9134
:1007E000FF90EF90DF90CF90089580E0F5CFCF930A
:1007F000DF93D82FC62FBFDE82E06EDC8D2F6CDC3E
:100800008C2F6ADCDF91CF9156CDFF920F931F930F
:10081000CF93DF93C82FF62E172F042FACDE83E083
:100820005BDC8C2F59DCCF2DD12F0C0F1D2F111D10
:10083000C017D10721F080E04FDC8993F9CFDF9119
:10084000CF911F910F91FF9036CDBF92CF92DF9243
:10085000EF92FF920F931F93CF93DF93CDB7DEB745
:100860002597CDBFDEBF8C01000F111F000F111F98
:10087000F801EC57FE4A45E0BE016F5F7F4F818172
:10088000C4DF8A81C98098E0C99E60011124282FA5
:1008900030E055E0359527955A95E1F7C20ED31E05
:1008A0000D2C000CEE08FF0883FF20C092E0CC0C5A
:1008B000DD1CEE1CFF1C9A95D1F78370C80ED11C6D
:1008C000E11CF11CFE2CED2CDC2CCC248B81C80E01
:1008D000D11CE11CF11CFE2CED2CDC2CCC248C81D9
:1008E000C80ED11CE11CF11C6894F7F88D818F7043
:1008F000B82EE8E081E090E0EB1510F1F801EC573C
:10090000FE4A80812BDF83FF02C06894F6F8C09214
:10091000303CD092313CE092323CF092333CB09289
:10092000343C0C571E4A4B2D68E37CE3F80182816E
:100930006CDF40E0F80163818CE2FDDE90E080E056
:100940002596CDBFDEBFDF91CF911F910F91FF9014
:10095000EF90DF90CF90BF900895CF92DF92EF920B
:10096000FF920F931F93CF93DF93CDB7DEB72D97F1
:10097000CDBFDEBF8091303C9091313CA091323CA4
:10098000B091333CAC01BD01442777FD4395552719
:10099000662777276C017D01CC24DD24EE2420E43A
:1009A000F2220FEF1FEF2FEF3FE1411104C00FEFD5
:1009B00017E020E030E080239123A223B3234423D7
:1009C00009F442C08C839B83CD01AA27BB27282F23
:1009D00023702860382F330F330F330F307E232BD3
:1009E0002A8335E0969587953A95E1F789831091AA
:1009F000343C812FCD28CE28CF2809F080648D8308
:100A0000412F50E068E37CE3CE01069658D345E0E1
:100A1000410FBE016F5F7F4F81E46EDE48E068E00A
:100A200080E489DE80E49ADE8077E1F084E090E083
:100A30002D96CDBFDEBFDF91CF911F910F91FF901B
:100A4000EF90DF90CF9008959C0193E03695279525
:100A50009A95E1F729838295880F807E8A831C828C
:100A60001B82C5CF90E080E0E3CF1F920F920FB6BC
:100A70000F9211248F939F93AF93BF9380912B3C40
:100A800090912C3CA0912D3CB0912E3C0196A11D43
:100A9000B11D80932B3C90932C3CA0932D3CB093A4
:100AA0002E3C81E08093A60ABF91AF919F918F91D8
:100AB0000F900FBE0F901F901895E0E4FCE384E0C8
:100AC000818381E38083E2E4FCE3158214823CDBD2
:100AD00083E08093813C61E009DBEDCBCF93DF9332
:100AE000CDB7DEB7A297CDBFDEBF91E088ED84BF62
:100AF0009093610080910206856080930206809148
:100B00000006816080930006809102068F7C8065DC
:100B1000809302061092E20582E08093E4059093B0
:100B2000030A8EEF8093270A8093260A80E8809339
:100B30002D0A80932B0A8093290A80932C0A809394
:100B40002A0A8093280A89E08093000A87E080932C
:100B5000E505E0E8FAE017E09EEF80E805E01183A4
:100B60009487858700837096E03C2AE0F207B9F706
:100B70001092A10A8FE39FE18093AC0A9093AD0A93
:100B80008091A50A81608093A50A1092A00A8091A5
:100B9000A00A81608093A00A7894D6DA85E190E07B
:100BA0008093033C9093043C81E08093053C8093C8
:100BB000063C8093073C26E130E02093083C3093CC
:100BC000093C80930A3C80930B3C92E090930C3C50
:100BD00027E130E020930D3C30930E3C80930F3C96
:100BE0008093103C93E09093113C28E130E02093F7
:100BF000123C3093133C8093143C8093153C94E05A
:100C00009093163C2CE130E02093173C3093183C35
:100C10008093193C80931A3C00931B3C2BE130E0FD
:100C200020931C3C30931D3C80931E3C80931F3CC2
:100C300096E09093203C2AE130E02093213C3093D1
:100C4000223C8093233C8093243C1093253C29E153
:100C500030E02093263C3093273C8093283C8093BF
:100C6000293C88E080932A3C80916000806890E075
:100C700028ED24BF809360007EDC80EC2DDA1BDB46
:100C80006AE070E080E090E0EBDB8E010F5F1F4FC9
:100C90008EE0F80111928A95E9F74EE0B80180E301
:100CA0002BDD4EE0B80180E427DD4EE0B80180E5A1
:100CB00023DD60E080E69BDD60E080E798DD63EAAD
:100CC0008BE295DD44E067E680E635DD41E067E6EE
:100CD00080E731DD8CE0E4EDF0E5DE011F96019068
:100CE0000D928A95E1F75E01FFE0AF0EB11CD12CA9
:100CF000C12CB8E09B2EF501019111915F0180E8B4
:100D00003BDD892B71F40230110509F475C108F03F
:100D10002CC10115110509F434C10130110509F484
:100D200071C180E829DD892B49F460E08AE25FDD4A
:100D300060E989E25CDD62E888E259DD80E01CDD83
:100D4000FBE2CF2EFCE3DF2E03E01CE3F801808101
:100D5000893210F462E0CAD9C801AEDBF80182839F
:100D60000B5F1F4FC016D10689F750910311909168
:100D70000511409107113091091120910B11892F14
:100D8000880F811D880F8527942F990F911D990F2A
:100D9000911D8927932F929590FB979597F9892715
:100DA000922F929589278093003C50910411409195
:100DB00006113091081120910A1190910C11440FE5
:100DC000411D440F4527330F311D330F311D43277C
:100DD000229520FB279527F9422792954927409392
:100DE000013C90E0982F8827092E000CAA0BBB0B22
:100DF00050E070E060E06F6F7F68842B952BA62B2E
:100E0000B72B8093303C9093313CA093323CB0930D
:100E1000333C84E08093343C81E08093383C1092F2
:100E2000393C82E080933A3C10923B3C96DD992419
:100E3000939465E0862E70E0A72E70E0B72EE2E076
:100E40007E2E33E0C32E3CE3D32EF601838188232C
:100E5000C1F1C60131DBF6019281891791F16AE097
:100E600070E080E090E0FCDAC60126DBF6019281BA
:100E7000891739F1828394814091003C50E0542FCE
:100E80004427052E000C660B770B2090013C312C7B
:100E9000512C412CF0E54F2A689457F842295329E8
:100EA000642975294093303C5093313C6093323C27
:100EB0007093333C7092343C9093383C8093393C2F
:100EC0004CDD25E0C20ED11CC016D10609F0BDCF05
:100ED00052DB80EA01D980E0FFD8D82EECD990E02F
:100EE00080E0D0FC04C0D1FE35C081E090E0ADDCF4
:100EF000892B81F58091023C89258093023C2091C9
:100F0000383CDD24D3948091393C811101C0D12C2F
:100F1000E3E0FCE390E080E03481231384C0889E0A
:100F20009001899E300D1124C9018D5F934C7C0185
:100F3000F7018381882339F08081893210F461E0E0
:100F4000D5D8F7011382F701D2828081893210F45B
:100F50006D2D73D964E170E080E090E081DAA11436
:100F6000B10409F46ECF4CD86CCF0430110509F4EC
:100F700047C008F443C00530110509F0D2CE88E11E
:100F800001C080E0F1E0CF16D104F1F51E8E1D8E78
:100F90009C8E1B8E44E0BE01655E7F4FADDB2FEF64
:100FA000C21AD20A86E0C816D10409F0A4CE1F8E58
:100FB00018A281E090E089A39AA38E01015E1F4FE1
:100FC0005E0193E2A90EB11CA8E09A2EF801C1902F
:100FD000D1908F0180E8D0DB892B09F0A2CE1E8E44
:100FE0001D8E9C8E1B8EC114D10499F0CA94CD28FD
:100FF00009F097CE84E20EC088E0C4CF80E1C2CF72
:1010000084E1C0CF84E0BECF1B8E1C8E1E8E1D8E51
:10101000C1CF80E244E0BE01655E7F4F6DDB0A1503
:101020001B05A1F67ECE019635968830910509F014
:1010300073CF7ECF38D0A59F900DB49F900DA49F05
:10104000800D911D1124089597FD1094002E0830F5
:1010500098F00850232F342F452F562F672F782FC5
:10106000892F912DF4CF159497958795779567954E
:1010700057954795379527950A95AAF71124002D7E
:1010800008950024A7FD00942A1730054005500557
:1010900060057005800590050895EE0FFF1F05900F
:1010A000F491E02D0994A29FB001B39FC001A39FCA
:1010B00001D0B29F700D811D1124911D0895FB0177
:1010C000DC0102C001900D9241505040D8F70895C4
:0410D000F894FFCFC2
:1010D40000000100020003000400050000000000FD
:1010E40000000000000000000005010101010101F1
:1010F40000000000000000000000000000000000EC
:1011040000000203000001020304050607000102B7
:101114000304050001020304050607000102030499
:10112400050607000102030001020304050600008E
:10113400000000000000010101010101020202029D
:10114400020202020303030303030303040404046B
:101154000505050505050501020408102040800168
:101164000204081020010204081020408001020437
:1011740008102040800102040801020408102040E5
:081184006061660170717602E2
:00000001FF
